:1012BF002321323030454655002324323030454605
:0212CF005500C8
:10128000AF8475840F758A83E4F597F58475C0443F
:0712900075CFE4C2C38F8497
:011297002234
:0D1053009000F1EFF09000F0E0FFA3E0FD51
:05106000900142EDF0DB
:1010650012115CEFC454F0900143F0900142E0FF8F
:0B10750012115C900143E02FF0E0FF3F
:01108000224D
:101081008F828E83D3E5829DE5839C501943B701FE
:10109100758F03E4F0F58F53B7FE2582F582740452
:0610A1003583F58380DEBB
:0110A7002226
:050C7400900136EFF0D5
:100C790020C3FD20C5FAC2C4D2C5E4FFFE30C3FDBE
:100C890030C3FDE5C154F8FC64086004ECB41016E7
:100C9900EF90013AB40105E044018003E054FEF508
:100CA900C27E01020D3FECB4180E900139E0F5C285
:100CB9007E02C2C4C2C5807EECB420028042EC64CC
:100CC900287039900136E06401700DEEB40202809B
:100CD90017EE64047022801CEEB402088BC27E03F6
:100CE900C2C58014EEB403088DC27E04C2C5800853
:100CF900EEB40404D2C57F01C2C4803AECB4300A10
:100D0900D2C4D2C57E09E4FF802CECB4380280221B
:100D1900ECB44006C2C2C2C5801CECB448028012C1
:100D2900ECB450028004ECB45808D2C47E08A9C2BD
:100D39008004D2C4D2C5C2C3EE64086003020C8920
:020D4900AF01F8
:010D4B002285
:10129800AE05AD07900139EEF0A3EBF0E4FB7F015A
:0412A800120C74228E
:10121C00AE03AC05AD07AF04AB07900139EEF0A3FC
:09122C0074A0F07F02120C742280
:0609F5009001161209C674
:1009FB007BFF7A1279BF9001201209C67B017A0026
:100A0B00790890011D1209C6900119120975000091
:100A1B000000E47F50FEFDFC900119120928C3125F
:100A2B0008E0503290011912091C7BA0E4FD121250
:100A3B009890011DE475F0011209AFEF12089E901A
:100A4B00011912091CE47B01FAF9F81208C690018E
:100A5B001912096980BC9001201209A6120858FFCF
:100A6B00900008E06F7068900001120871FF900011
:100A7B0009E06F705A900002120871FF90000AE0B3
:100A8B006F704C900003120871FF90000BE06F70B9
:100A9B003E9001201209A6900004120871FF9000ED
:100AAB000CE06F702A900005120871FF90000DE0AA
:100ABB00B5071C900006120871FF90000EE0B507F9
:100ACB000E900007120871FF90000FE06F60037F1C
:100ADB0000229001161209A6120858FF900019E087
:100AEB006F702A900001120871FF90001AE0B50791
:100AFB001C900002120871FF90001BE0B5070E90CE
:100B0B000003120871FF90001CE06F60037F00224E
:100B1B00900011E0900004F0900012E0FFA3E09031
:100B2B000006CFF0A3EFF0900021E0900000F090D2
:100B3B000022E0FFA3E0900002CFF0A3EFF07F01D3
:010B4B002287
:1010F40090010AEFF0900114E0FEA3E0FF12124EFB
:08110400900114EEF0A3EFF0DE
:0A110C00EEFD900001E0FB121298C6
:0111160022B6
:10123500900004E0FFA3E0C39F500D900001E0245F
:0912450002F0900005E004F02223
:10124E000FBF00010EC3900007E09F900006E09EC6
:09125E005006121235E4FEFF22D5
:08069300900107EEF0A3EFF067
:10069B00E490010AF0A3F0900110F0A3F0A3F0A3F3
:1006AB00F0A3F0A3F0900002E0FFA3E0900114CFC1
:1006BB00F0A3EFF0900000E0A3F0E490010BF090BA
:1006CB00010AF090000504F0E490010FF090010A8C
:1006DB00E0643A6025900114E0FEA3E0FF12110CD8
:1006EB0090010AEFF0900114E0FEA3E0FF12124E0E
:1006FB00900114EEF0A3EFF080D3900110E475F0AD
:10070B00011208B0900114E0FEA3E0FF12110C12CD
:10071B0010F490010BEFF0FD90010AE0FF12106056
:10072B0090010DEFF090010F1210F81210F49001E0
:10073B000BEFF0FD90010AE0FF121060900112E444
:10074B00F0A3EFF0900112A3E0FFFD90010FE02D5D
:10075B00F0EF900112F0A3E4F0A31210FC1210F4CE
:10076B0090010BEFF0FD90010AE0FF121060900179
:10077B0012E0FEA3E04FFF900112EEF0FEA3EFF0AC
:10078B00AC068C12F51390010FE02F1210F812101B
:10079B00F490010BEFF0FD90010AE0FF1210609056
:1007AB00010CEFF090010FE02FF0EF707590010945
:1007BB00F090010DE0FF900109E0C39F506412100F
:1007CB00F91210F490010BEFF0FD90010AE0FF120B
:1007DB00106090010EEFF0A3E02FF0D3900108E032
:1007EB009513900107E09512502FAE12AF13BEFB7D
:1007FB0006BFFE0343B13043B701758F0190010E65
:10080B00E0851382851283F0E4F58F53B7FE75B143
:10081B00110513E51370020512900109E004F002B3
:10082B0007BC1210F91210F490010BEFF0FD9001C0
:10083B000AE0FF12106090010EEFF0A3E02F700C96
:0C084B0090010CE0640160030206D3225F
:01085700227E
:060B4C009001231209C60E
:100B52007BFF7A1279C890012D1209C67B017A00B7
:100B6200795890012A1209C69001261209750000CF
:100B72000000E47F2BFEFDFC900126120928C3121F
:100B820008E0503190012612091CE4FBFD12121CF0
:100B920090012AE475F0011209AFEF12089E90014C
:100BA2002612091CE47B01FAF9F81208C690012604
:100BB20012096980BD90012D1209A6120858FF90F2
:100BC2000058E06F7068900001120871FF900059A0
:100BD200E06F705A900002120871FF90005AE06FA5
:100BE200704C900003120871FF90005BE06F703E42
:100BF20090012D1209A6900004120871FF90005C6A
:100C0200E06F702A900005120871FF90005DE0B558
:100C1200071C900006120871FF90005EE0B5070EF7
:100C2200900007120871FF90005FE06F60037F0081
:100C3200229001231209A6120858FF900067E06F64
:100C4200702A900001120871FF900068E0B5071C3D
:100C5200900002120871FF900069E0B5070E900043
:100C620003120871FF90006AE06F60037F00227F29
:010C72000180
:010C7300225E
:0B0FAB009000F0EFF09000FF120934FE
:060FB60090013B120969E5
:100FBC0090013B12091CAB0790013B12091C7808ED
:100FCC001208F6AA0790013B12091C78101208F6B9
:0B0FDC00AE07AF03AD02AB0612121C03
:010FE70022E7
:08040B009000EDEEF0A3EFF00C
:10041300E49000F0F0A3F09000FB120975000000D7
:10042300009000FF120975000000009001031209FB
:1004330075000000009000FF1209750000002BE416
:100443009000F1F09000F0F09000F6F0E49000F5E9
:10045300F09000F0E0643A600A120FB09000F0EF01
:10046300F080EE90010312091CEF2401FFE43EFE2D
:10047300E43DFDE43CFC900103120969120FB01244
:100483000FAB1210539000F3EFF09000F5120FAF83
:10049300120FAB121053E4FCFDFE9000F712096932
:1004A3009000F712091C9000F5E02FF09000F7126E
:1004B300091C78081209099000F7120969120FB094
:1004C300120FAB9000F1EFF09000F7120928C00073
:1004D300C001C002C003121058E4FCFDFED003D0DB
:1004E30002D001D0001208D39000F71209699000DE
:1004F300F712091C8E148F159000F712091C900037
:10050300F5E02F120FAF120FAB1210539000F2EF62
:10051300F09000F5E02FF0EF64047066120FB01254
:100523000FAB121053E4FCFDFE9000FB120969901F
:1005330000FB12091C78081209099000FB120969D3
:10054300120FB0120FAB9000F1EFF09000FB120905
:1005530028C000C001C002C003121058E4FCFDFE15
:10056300D003D002D001D0001208D39000FB1209AF
:10057300699000FB12091C78101209099000FB1204
:1005830009699000F2E064027066120FB0120FABBB
:10059300121053E4FCFDFE9000FB1209699000FB6E
:1005A30012091C78081209099000FB120969120F3D
:1005B300B0120FAB9000F1EFF09000FB120928C0CE
:1005C30000C001C002C003121058E4FCFDFED003BA
:1005D300D002D001D0001208D39000FB1209699019
:1005E30000FB12091C78041209099000FB12096927
:1005F3009000FB12091CEF2515F515EE3514F514C3
:100603009000F2E0706A9000EFF09000F3E0FF904A
:1006130000EFE0C39F5059120FB0120FAB121053EB
:100623009000F4EFF0A3E02FF0D39000EEE09515E7
:100633009000EDE09514502FAE14AF15BEFB06BF2E
:10064300FE0343B13043B701758F019000F4E08599
:100653001582851483F0E4F58F53B7FE75B1110548
:1006630015E515700205149000EFE004F002060D85
:10067300120FB0120FAB1210539000F4EFF0A3E07F
:0F0683002F700C9000F2E06401600302044F221C
:010692002245
:10117E00436865636B20666F72006669726D776196
:0F118E00726520757064617465003239314500F7
:100EC300AE8475840F758A83E4F59775840FF5896D
:100ED300F58475B73075840F4389018D8D758F0146
:100EE3008F8EFDFC0DBD00010CE4B505F7ECB401DC
:100EF300F3438902E58920E4120DEDAA0470010C85
:100F030014D39400EA6480948140E9759702AF0694
:020F13008F84C9
:010F150022B9
:10111700AF8475840F75E10343E20443E3C075A40C
:101127000F7580F075A51775AD17E4F5A675A7F0CF
:021137008F84A3
:011139002293
:1012AC00AF84E4F584759D0443F808759A40D2F830
:0212BC008F841D
:0112BE00220D
:0612EE001212800212AC96
:100E0B00C20CE4FFFEE4900144F0A3F0900144E433
:100E1B0075F0011208B0900144E0B403EFA3E0B405
:100E2B0020EA0FBF00010EBE0BDBBFB8D81211BCFE
:100E3B00E4900144F0A3F0120F66EF64134E7004BC
:100E4B00D20C8019900144E475F0011208B0C390E4
:0F0E5B000145E094FB900144E0940940DAA20CB9
:010E6A002265
:100D4C00C209C20AC20B75FFDE75FFAD7D017F04BF
:100D5C00120EC31211171212D17BFF7A11797E90E9
:100D6C0000861209C67B017A0079AB12010B7BFF5E
:100D7C007A1179889000861209C67B017A0079BCB9
:100D8C0012010B7B017A0079BC9001331209C67AEF
:100D9C000079AB120E6B120E0B920930095E121217
:100DAC00EE7BFF7A1179981209F5EF24FF920A3045
:100DBC000A147D007CCC7F007E401210817F007E67
:100DCC004012069380237BFF7A117998120B4CEF1B
:100DDC0024FF920B300B127D007CCC7F007E4012E6
:100DEC0010817F007E4012040BE4FFFE0FBF000158
:0F0DFC000EBE27F8BF10F5E4F584F5C002000E17
:04000E00024000228A
:1012D1007F3812119D7F0612119D7D0EE4FF0211D0
:0112E100F319
:05119D00900146EFF097
:1011A200A2AF920DC2AF12113AEF20E7F9900146B9
:0911B200E0FF120FE8A20D92AF5C
:0111BB002211
:10113A00A2AF920EC2AF75A0FFC2B6D2B5D2B77F28
:10114A0014DFFEAEA0C2B77F14DFFEA20E92AFAFCD
:01115A00068E
:01115B002271
:050006007F0102119DC5
:100FE800A2AF920FC2AF8FA07F147E00EF1F7001D7
:100FF8001EEF4E70F7C2B6C2B5D2B77E007F14EFAF
:101008001F70011EEF4E70F7C2B77E007F14EF1FEE
:0B10180070011EEF4E70F7A20F92AFA8
:0110230022AA
:10102400A2AF9210C2AF8FA0C2B5D2B7D2B67F140E
:101034007E00EF1F70011EEF4E70F7C2B77E007F77
:0E10440014EF1F70011EEF4E70F7A21092AF56
:01105200227B
:0C11F300900147E05FF04DFFF002119DFD
:02126700AD07D1
:10126900A2AF9211C2AF12113AEF20E7F9AF0512FE
:061279001024A21192AF47
:01127F00224C
:1010CF0090013F1209C690013F1209A612085860FD
:1010DF001390013FE475F0011209AF120858FF1287
:0510EF00126780E222FF
:060E6B009001301209C6DF
:100E7100A2AF9212C2AF120006A21292AFC2AFE4A9
:100E8100FDFF1212E2A21292AFC2AF90013012091D
:100E9100A61210CFA21292AFC2AFE4FD7F011212CF
:100EA100E2A21292AFC2AF9001331209A61210CF83
:100EB100A21292AFC2AF7D117F011212E2A2129271
:010EC100AF81
:010EC200220D
:0C12E200EF75F040A42D2480FF02119D48
:1011BC007F209000CDE4F0A3DFFC7B017A0079CD99
:0C11CC008B0A8A0B890C8A088909D2B4AE
:0111D80022F4
:100F6600AF8475840FE5B0540FFEE58054801313EB
:100F760013541F4EFE0509E509AC08700205081456
:100F8600F5828C83EEF0C3E50994EDE50894004004
:100F9600067508007509CDC2B43086FDD2B48F84BB
:040FA600AF067E0014
:010FAA002224
:01FBFE00FE08
:030000000211D911
:03000300025003A5
:03000B000250069A
:030013000250098F
:03001B0002500C84
:0300230002500F79
:03002B000250126E
:0300330002501563
:03003B0002501858
:0300430002501B4D
:03004B0002501E42
:0300530002502137
:03005B000250242C
:0300630002502721
:03006B0002502A16
:0300730002502D0B
:03007B0002503000
:03008300025033F5
:03008B00025036EA
:03009300025039DF
:03009B0002503CD4
:0300A30002503FC9
:1011D900787FE4F6D8FD9000007F007E20E4F0A33C
:0A11E900DFFCDEFA758122020D4CD6
:100F1600E590540C23C0E07412C0E0C082C0830286
:100F26001200E590540C23C0E07412C0E0C082C0E9
:100F360083021208E590540C23C0E07412C0E0C08E
:100F460082C083021210E590540C23C0E07412C0D4
:080F5600E0C082C08302121802
:041200005390F322F2
:0712080043900C5390F72204
:0712100043900C5390FB22F8
:0412180043900C22D1
:070F5E00EFC40390120073C1
:10085800BB010689828A83E0225002E722BBFE029E
:09086800E32289828A83E49322D1
:10087100BB010CE58229F582E5833AF583E022503C
:1008810006E92582F8E622BBFE06E92582F8E22286
:0D089100E58229F582E5833AF583E49322A0
:10089E00BB010689828A83F0225002F722BBFE0139
:0208AE00F32233
:1008B000C5F0F8A3E028F0C5F0F8E58215827002D3
:0608C0001583E038F02270
:0D08C600EF2BFFEE3AFEED39FDEC38FC2281
:0D08D300EF4BFFEE4AFEED49FDEC48FC2224
:1008E000EB9FF5F0EA9E42F0E99D42F0EC6480C88F
:0608F00064809845F0222F
:1008F600E8600FECC313FCED13FDEE13FEEF13FFE0
:03090600D8F12203
:10090900E8600FEFC333FFEE33FEED33FDEC33FC4C
:03091900D8F122F0
:0C091C00E0FCA3E0FDA3E0FEA3E0FF224E
:0C092800E0F8A3E0F9A3E0FAA3E0FB2252
:100934007401FF3395E0FEFDFCA3A3A3E0CF2FF0E9
:10094400E582158270021583E0CE3EF0E5821582C1
:1009540070021583E0CD3DF0E582158270021583A7
:05096400E0CC3CF02294
:0C096900ECF0A3EDF0A3EEF0A3EFF02201
:10097500A8828583F0D083D08212098C12098C124B
:10098500098C12098CE473E493A3C583C5F0C58370
:10099500C8C582C8F0A3C583C5F0C583C8C582C8CC
:0109A500222F
:0909A600E0FBA3E0FAA3E0F92252
:1009AF00F8E0FBA3A3E0F925F0F0E58215827002D1
:0709BF001583E0FA38F02275
:0909C600EBF0A3EAF0A3E9F02232
:1000A600E50D2486F582E43400F583E0050D229003
:1000B6000083300703900086E475F0011209AF0251
:1000C60008582000E97F2ED2008018EF540F2490A4
:1000D600D43440D4FF30040BEF24BFB41A005003CD
:1000E6002461FFE50E6002150E0511E5117002058B
:1000F6001030070E900083E475F0011209AFEF028D
:10010600089E0210A87403D2078003E4C207F50D07
:100116009000831209C6E4F50EF510F511E50E60A0
:10012600077F201200E980F5750FFFC201C200C2E9
:1001360002C203C205C206C2081200B5FF700D3026
:1001460007057F001200FAAF11AE1022B4255FC278
:10015600D5C2041200B5FF24D0B40A00501A75F0B7
:100166000A780E30D50508B6FF0106C6A426F62085
:10017600D5047002D20380D924CFB41A00EF5004FC
:10018600C2E5D2040202FBD20180C6D20080C0D2F0
:100196000280BCD2D580BAD20580B47F201200E995
:1001A6002002077401B50E0040F11200A6FF1200EE
:1001B600E9020123D208D20680951200A6FB12009E
:1001C600A6FA1200A6F94A4B700679CC7A037BFF91
:1001D60020022EE50E602A7E008E827583001208AC
:1001E6007160060EEE650F70F0C2D5EBC0E0EAC096
:1001F600E0E9C0E0EE120342D0E0F9D0E0FAD0E048
:10020600FB120858FF60AAEBC0E0EAC0E0E9C0E0D4
:100216001200E9D0E02401F9D0E03400FAD0E0FB86
:10022600E50F0460DCD50FD980877BFF7A03793E22
:10023600D202809C791080027908C206C208800822
:10024600D2D5790A8004790AC2D5E50F047002F581
:100256000FE4FAFDFEFF1200A6FC7B082001131234
:1002660000A6FD7B1030000A1200A6FE1200A6FFB3
:100276007B20EC3382D592D55013C3E43000069F21
:10028600FFE49EFEE42001039DFDE49CFCE4CBF824
:10029600C201EC700CCFCECDCCE824F8F870F38018
:1002A60017C3EF33FFEE33FEED33FDEC33FCEB33D8
:1002B600FB994002FB0FD8E9EB300105F8D0E0C40A
:1002C60048B201C0E00AEC4D4E4F78207B0070C268
:1002D600EAB50F0040BCC0E0120344D0F0D0E020E5
:1002E6000104C4C0E0C4B201C0F01200D2D0F0D5FF
:1002F600F0EB0201231209CF01C053023A580191D3
:100306004C018D42023E4F02464402464901A64335
:08031600024C55023046023092
:10031E004502304703EC5001952D01992E01BC2B5F
:10032E00019D2301BA2003D52A015548000001B4CE
:10033E003F3F3F00790AA2D5200314300509B910BA
:10034E00020404B9080104A2D520060250010420BB
:10035E0002689202B50E005034C0E07F20300319BF
:10036E007F30A20272067205500F12039BC202C2A8
:10037E0006C205C2087F30800F300503E9C0E012C7
:10038E0000E9300503D0E0F9D0E0B50ECC3005170A
:10039E007F30B9100C1200E97F583004077F788047
:1003AE0003B908031200E93002057F2D0200E97F30
:1003BE00202008F87F2B2006F322920280CF286E91
:1003CE00756C6C2900D2011200A63001F8C20178BA
:1003DE000E30D50108F60201552D50434958120032
:1003EE00A62403B405004001E49003E7931200DA5B
:0D03FE00743A1200DAD203750E0402023ABE
:10115C00EF7E0024D0B40A00401624F9B40A0040F3
:10116C000CB41000400A24E0B41000400374FFFEDD
:02117C00FF2250
:1009CF00D083D082F8E4937012740193700DA3A3B7
:1009DF0093F8740193F5828883E4737402936860CB
:0609EF00EFA3A3A380DFCB
:1010A800EFB40A07740D1210B3740A309811A89996
:1010B800B8130CC2983098FDA899C298B811F630A8
:0710C80099FDC299F5992280
:00000001FF
